:100000000C942A000C9445000C9445000C94450077
:100010000C9445000C9445000C9445000C9445004C
:100020000C9445000C9445000C9445000C9447003A
:100030000C9445000C9445000C9445000C9445002C
:100040000C94BC000C9445000C9445000C944500A5
:100050000C94450011241FBECFE5D8E0DEBFCDBF14
:1000600010E0A0E6B0E0E6ECF1E002C005900D92F1
:10007000A036B107D9F710E0A0E6B0E001C01D92AC
:10008000A537B107E1F70C948D000C9400001F9286
:100090000F920FB60F9211248F939F93809173004C
:1000A000982F9F5F90937300992321F4C09AC19A6F
:1000B000C29AC39A80916000981709F4C098809101
:1000C0006100981709F4C19880917400981709F499
:1000D000C29880917200981709F4C3989F918F91EC
:1000E0000F900FBE0F901F90189581E083BF89B7C6
:1000F000816089BF08958CEC86B980E090E022E6AB
:1001000030E0FC01EE0FFF1FE20FF31F118210829F
:10011000019688309105A9F70895CFE5D8E0DEBFB4
:10012000CDBF1ABA8FE087BB14BA11BA80E48093AE
:1001300060001092610010927400109272000E9490
:100140007B000E947500789480916200909163001A
:1001500099230CF4039695958795959587958093AB
:100160006000F2CFFC01E770F070EE0FFF1FEE5958
:10017000FF4F8081918108951F920F920FB60F92C9
:1001800011242F933F938F939F93EF93FF9387B106
:1001900099278770907024B135B1FC01EE0FFF1FD5
:1001A000EE59FF4F318320830196877087B9369AC5
:1001B000FF91EF919F918F913F912F910F900FBEE3
:0601C0000F901F9018953E
:00000001FF
